:020000040000FA
:06000000B7EF00F0120052
:02002A000000D4
:04002C002A0EF66E34
:10003000000EF76E000EF86E00010900F550656FB6
:100040000900F550666F03E1656701D03DD00900F6
:10005000F550606F0900F550616F0900F550626F4F
:1000600009000900F550E96E0900F550EA6E090033
:1000700009000900F550636F0900F550646F09002D
:100080000900F6CF67F0F7CF68F0F8CF69F060C0ED
:10009000F6FF61C0F7FF62C0F8FF0001635302E1A1
:1000A000645307E00900F550EE6E6307F8E2640759
:1000B000F9D767C0F6FF68C0F7FF69C0F8FF000115
:0A00C0006507000E665BBFD7120053
:0600CA001200D9CFE6FF91
:1000D000DACFE6FFE1CFD9FFE2CFDAFFE652E65210
:1000E000D9CFE9FFDACFEAFFEE6AED6A6E0EE66E6F
:1000F000A0EC00F0E552809280806E0EE66EA0ECDF
:1001000000F0E55280908082D9CFE9FFDACFEAFF94
:10011000EE2A000EEF22EAD7D8DF929092928092D8
:1001200080902C0EE66EA0EC00F0E552809280806C
:100130002C0EE66EA0EC00F0E55280908082F1D7A4
:10014000FF0EE350036EEF0E01D0F30EE76EE72EC5
:10015000A7EF00F00C0E026EE76AE72EADEF00F09D
:0E016000022EACEF00F0032EA5EF00F012000F
:02016E0011EE90
:1001700000F021EE00F0F86A019C16EC00F0CCECE7
:0A01800000F08CEC00F0FBD7120039
:06018A0000EE00F00F0E74
:08019000EE6AEA62FDD71200DD
:02019800120053
:020000040030CA
:010003001EDE
:00000001FF
